:020000040000FA
:10000000831307309F008501860183169F018501B8
:10001000FB308600811718121815193099009816B0
:10002000831298171816B2202830CF20A201A901F8
:10003000AA01AB01AC010030CF20BD20DC201B2881
:100040000C1E2028990008008C1E24281A08181954
:100050002B28981C08001812181624283830840001
:1000600000082F3A031D12293030840003100008C5
:10007000303A031940280008313A031D12290314AD
:10008000A30D840A00082F3A031D36282308A20076
:10009000850008006320A808031D1229A204220875
:1000A000850008006320A808031D1229FF3AA20555
:1000B0002208850008006320A808031D1229A20653
:1000C000220885000800840A00088A20A808031D69
:1000D000080009302602031C6F28A80A0800003017
:1000E0008A0026088207FF340134023404340834BD
:1000F0001034203440348034A60082202508A40027
:10010000A60E82280F302605F63E0318073E3A3E1B
:10011000A5000800A801A400463C031CA02841300B
:100120002402031C96280A3EA60008002408393C35
:10013000031CA02830302402031CA028A6000800BD
:10014000A80A080024088A20A808031D0800260E13
:10015000A70025088A20A808031D08002608A70470
:10016000A70E0800FF30AE00AD01AD030319BA2899
:10017000BC20B528AE0BB42808002F308400242002
:1001800080000D3A0319CD2800082020840A0408B5
:100190003A3A031DBF282F30840080010800A100D7
:1001A000782100380319080020200D3A031DDA28B1
:1001B0000A302020A10AD0282F3084000008031D17
:1001C000E22808006E30000603194A28663000064F
:1001D000031952287430000603195B287630000694
:1001E00003191529693000060319512963300006E7
:1001F00003195B296F300006031943296D3000068F
:1002000003191829703000060319252977300006D4
:10021000031932297330000603192E2852300006C4
:10022000031900280430CF2008004C30CF200800EC
:10023000840A69300006031D1F29A90908006F30D0
:100240000006031D1229AA090800840A6930000665
:10025000031D2C29AB0908006F300006031D12296D
:10026000AC090800840A65300006031D3B2983168B
:1002700081138312080064300006031D12298316BF
:100280008117831208004A30CF2018302C18CF2055
:1002900022082A186B297C202508202024082020E9
:1002A00008004A30CF2008302B18CF200608F83934
:1002B00029186B294B294A30CF200030013E031DFD
:1002C0005E2953210D3020208C1E5D2924202E3ADA
:1002D000031D5D290800A6000314A60D3030031885
:1002E000313020200310A60DA608031D6E2908003A
:0802F00003308A00210882009E
:100600000D342334203400340D343F34203400348E
:1006100049346E3470347534743420347334743423
:10062000613474347534733420343A3420340034F3
:100630004F347534743470347534743420347334F6
:10064000743461347434753473343A34203400347F
:100650000D345034493443342034533465347234C7
:10066000693461346C34203449344F342034633479
:100670006F346E34743472346F346C346C3465346B
:1006800072342034723465346134643479340D3416
:100690000A3400340D3400340D34463457342034D9
:1006A000563432342E3431342034323430342F3412
:1006B000303433342F3432343034303435340D3434
:0406C00000340034CE
:02400E00103F61
:00000001FF
